:0500000002003381370E
:02000B0081383A
:02001300813931
:02001B00813A28
:02002300813B1F
:02002B00813C16
:10003300759840758780758921758DFF758BFF7560
:100043008840D2997581607530007531007535FF30
:1000530075460075470AC2B4D2B575487F75497FA6
:10006300754A0F754B0A754C7F754D7F754E0F752D
:100073004F0875500F755109755211755308D210F9
:10008300D211D212D213D214D215D216D217D21839
:10009300D219D21AD21BD21CD21DD21ED21FD220E9
:1000A300D221D222D223D234D235D236D237C23859
:1000B300C239C23AC2B0D2A27407B535037535FF4F
:1000C3000535E535A2E092A4A2E192A5A2E292A6AB
:1000D300D2A7D290209014301021C210B211201157
:1000E300051204A880151204F2801020100DD210FE
:1000F3002011051204EE8003120538C2A7D2912005
:100103009114301221C212B21320130512053C8040
:1001130015120586801020120DD212201305120528
:100123008280031205CCD292209214301421C2147F
:10013300B2152015051205D0801512061A8010205D
:10014300140DD2142015051206168003120660D270
:1001530093209314301621C216B2172017051206E6
:100163006480151206AE801020160DD216201705D6
:100173001206AA80031206F4D29420941430182194
:10018300C218B2192019051206F880151207428009
:100193001020180DD21820190512073E80031207EC
:1001A30088D295209514301A21C21AB21B201B0540
:1001B30012078C80151207D68010201A0DD21A2030
:1001C3001B051207D2800312081CD2962096143006
:1001D3001C21C21CB21D201D051208208015120807
:1001E300528010201C0DD21C201D0512084E8003C6
:1001F300120880D297209714301E21C21EB21F20EE
:100203001F0512088480151208B68010201E0DD217
:100213001E201F051208B280031208E4D2A020A0FA
:1002230014302021C220B2212021051208E88015B4
:1002330012091A801020200DD22020210512091640
:100243008003120948D2A120A114302221C222B274
:100253002320230512094C801512097E80102022C9
:100263000DD22220230512097A80031209ACD2B2DF
:1002730020B214303421C234B2352035051209B00E
:1002830080151209C6801020340DD2342035051292
:1002930009C280031209D8D2B320B314303621C265
:1002A30036B2372037051209DC80151209F38010A6
:1002B30020360DD2362037051209EF80031209FAD2
:1002C300A23892B4B392B5D2B620B61975320712DA
:1002D30009FE12044CD53203753201120453D2B60F
:1002E30020B60280F0D2B720B719753207120A3050
:1002F30012044CD53203753201120453D2B720B71E
:100303000280F0E4B53502613204B535026152046E
:10031300B53502617204B53502619204B5350261E7
:10032300B204B5350261D204B5350261F28112E53A
:1003330080F536A837A93612045A400624FE500D1C
:10034300800512045F5006853637120A628132E552
:1003530080F538A839A93812045A400624FE500DF6
:10036300800512045F5006853839120A948132E5FC
:1003730080F53AA83BA93A12045A400624FE500DD0
:10038300800512045F5006853A3B120AC68132E5A6
:1003930080F53CA83DA93C12045A400624FE500DAA
:1003A300800512045F5006853C3D120AF88132E550
:1003B30080F53EA83FA93E12045A400624FE500D84
:1003C300800512045F5006853E3F120B2A8132E5F9
:1003D30080F540A841A94012045A400624FE500D5E
:1003E300800512045F5006854041120B848132E57B
:1003F30080F542A843A94212045A400624FE500D38
:10040300800512045F5006854243120BDE8132E5FC
:1004130080F544A845A94412045A400624FE500D11
:10042300800512045F5006854445120C0081320199
:10043300B7020033323232323232B2B4B2B57E2036
:10044300DFFEDEFCB2B4B2B5227E20DFFEDEFC228C
:100453007E60DFFEDEFC22C2D7E89922C2D7E9988C
:1004630024FE22B2B4B2B53099FDC2997599F03029
:1004730099FDC2997599423099FDC29975993030A9
:1004830099FDC2997599193099FDC29975994122BF
:100493003099FDC2997599003099FDC2997599F704
:1004A300B2B4B2B522D239D238D23A1204663099F4
:1004B300FDC29975990E3099FDC2997599083099C5
:1004C300FDC29975990A12049375487F75497F7522
:1004D3004A0F754B0A754C7F754D7F754E0F754FDF
:1004E3000875500F75510912043D2212044C22D293
:1004F30039D238D23A1204663099FDC29975990EF1
:100503003099FDC2997599083099FDC29975990A78
:1005130012049375487F75497F754A0F754B0A75A9
:100523004C7F754D7F754E0F754F0875500F755184
:100533000912043D2212044C22C239C23AD23812A3
:1005430004663099FDC29975990E3099FDC299756B
:1005530099083099FDC29975990012049375480F53
:1005630075490A754A0F754B0B754C7F754D7F7531
:100573004E0F754F0875500F75510912043D221225
:10058300044C22C239C23AD2381204663099FDC2F1
:100593009975990E3099FDC2997599083099FDC2E4
:1005A3009975990012049375480F75490A754A0F96
:1005B300754B0B754C7F754D7F754E0F754F0875D9
:1005C300500F75510912043D2212044C22C239C244
:1005D3003AD2381204663099FDC29975990E309952
:1005E300FDC2997599083099FDC29975990F120446
:1005F3009375480F75490B754A0F754B0A754C0F68
:10060300754D09754E0F754F0875507F75517F12E3
:10061300043D2212044C22C239C23AD23812046673
:100623003099FDC29975990E3099FDC29975990853
:100633003099FDC29975990F12049375480F754946
:100643000B754A0F754B0A754C0F754D09754E0F97
:10065300754F0875507F75517F12043D2212044C6B
:1006630022C239C23AD2381204663099FDC2997552
:10067300990E3099FDC2997599083099FDC2997503
:10068300990D12049375480F75490B754A0F754BF5
:1006930008754C0F754D09754E0F754F0A75507FD0
:1006A30075517F12043D2212044C22C239C23AD240
:1006B300381204663099FDC29975990E3099FDC2BE
:1006C300997599083099FDC29975990D120493751E
:1006D300480F75490B754A0F754B08754C0F754DCF
:1006E30009754E0F754F0A75507F75517F12043D82
:1006F3002212044C22C239C23AD23812046630990B
:10070300FDC29975990E3099FDC299759908309972
:10071300FDC29975990B12049375487F75497F75CE
:100723004A0F754B08754C0F754D09754E0F754F74
:100733000A75507F75517F12043D2212044C22C268
:1007430039C23AD2381204663099FDC29975990EAE
:100753003099FDC2997599083099FDC29975990B25
:1007630012049375487F75497F754A0F754B087559
:100773004C0F754D09754E0F754F0A75507F7551A6
:100783007F12043D2212044C22C239C23AD23812DB
:1007930004663099FDC29975990E3099FDC2997519
:1007A30099083099FDC29975991812049375487F79
:1007B30075497F754A0F754B08754C0F754D0A7552
:1007C3004E7F754F7F75507F75517F12043D221206
:1007D300044C22C239C23AD2381204663099FDC29F
:1007E3009975990E3099FDC2997599083099FDC292
:1007F3009975991812049375487F75497F754A0F47
:10080300754B08754C0F754D0A754E7F754F7F7587
:10081300507F75517F12043D2212044C22C239C20B
:100823003AD2381204663099FDC2997599103099FD
:10083300FDC2997599083099FDC2997599041204FE
:100843009375521175530812043D2212044C22C2AF
:1008530039C23AD2381204663099FDC2997599109B
:100863003099FDC2997599083099FDC2997599041B
:1008730012049375521175530812043D2212044C4D
:1008830022C239C23AD2381204663099FDC2997530
:1008930099103099FDC2997599083099FDC29975DF
:1008A300990012049375521175530812043D2212D4
:1008B300044C22C239C23AD2381204663099FDC2BE
:1008C300997599103099FDC2997599083099FDC2AF
:1008D3009975990012049375521175530812043DCA
:1008E3002212044C22C239C23AD238120466309919
:1008F300FDC2997599103099FDC29975990830997F
:10090300FDC29975990B120493755211755309120F
:10091300043D2212044C22C239C23AD23812046670
:100923003099FDC2997599103099FDC2997599084E
:100933003099FDC29975990B120493755211755331
:100943000912043D2212044C22C239C23AD238128F
:1009530004663099FDC2997599103099FDC2997555
:1009630099083099FDC29975991112049375521122
:1009730075530912043D2212044C22C239C23AD2E1
:10098300381204663099FDC2997599103099FDC2E9
:10099300997599083099FDC2997599111204937547
:1009A300521175530912043D2212044C22B238200D
:1009B3003804C2398005303A02D23912044C22126B
:1009C300044C22B238203804C2398005303A02D2AE
:1009D3003912044C2212044C2275470B12043D12A7
:1009E300044C12044C12044C12043D2212044C22F7
:1009F30075470A12043D2212044C22D2B4C2B5C276
:100A030039C23AD2381204663099FDC299759910E9
:100A13003099FDC2997599083099FDC2997599105D
:100A230012049375521175530912043D22D2B4C2B4
:100A3300B5C239C23AD2381204663099FDC29975EB
:100A430099103099FDC2997599083099FDC299752D
:100A5300990D12049375521175530912043D221214
:100A630004663099FDC29920380D8547993099FD68
:100A7300C29975990C800B854C993099FDC2998563
:100A83004D993099FDC299E536C313F59912049334
:100A9300221204663099FDC29920380D854799309A
:100AA30099FDC29975990A800B854A993099FDC2BF
:100AB30099854B993099FDC299E538C313F599127D
:100AC3000493221204663099FDC29920380D75995A
:100AD300033099FDC299759909800B85489930991E
:100AE300FDC2998549993099FDC299E53AC313F539
:100AF30099120493221204663099FDC29920380D8D
:100B03007599013099FDC299759908800B855299A1
:100B13003099FDC2998553993099FDC299E53CC33B
:100B230013F599120493221204663099FDC2992099
:100B3300380D7599073099FDC29975990E800B850B
:100B430050993099FDC2998551993099FDC29920E8
:100B5300390AE53EC313F59912049322E53EC31304
:100B6300F5F0541F2323F5993099FDC299E5F0540C
:100B7300600303030303F5993099FDC2997599F74F
:100B8300221204663099FDC29920380D75990730F9
:100B930099FDC299759908800B854E993099FDC2CC
:100BA30099854F993099FDC29920390AE540C313BD
:100BB300F59912049322E540C313F5F0541F232340
:100BC300F5993099FDC299E5F054600303030303DB
:100BD300F5993099FDC2997599F7221204663099F7
:100BE300FDC29975990F3099FDC29975990F309986
:100BF300FDC299E542C313F59912049322120466C8
:100C03003099FDC2997599113099FDC29975990F63
:100C13003099FDC299E544C313F599120493222038
:100C23004D757A796B616E7420352076312E30667E
:100C330020323030372D30332D3036202863294190
:100C430064616D20536D69616C656B206A616E6BC5
:100C53006F6D757A796B616E744077702E706C204E
:100C63007777772E736D69616C656B2E7072762E54
:100C7300706C2057737A656C6B696520707261774D
:100C830061207A617374727A657A6F6E652E204A79
:100C9300616B69656B6F6C7769656B207A617374DF
:100CA3006F736F77616E6961206B6F6D65726379C6
:100CB3006A6E65206B6F6475206E6965646F7A7701
:100CC3006F6C6F6E652E20416C6C2052696768747F
:100CD300732052657365727665642E20467265656E
:100CE30020666F72206E6F6E20636F6D6D65726329
:0A0CF30069616C206F6E6C792E2091
:00000001FF
